:020000040000FA
:100000008301022803138316FF3085000F3086001A
:10001000FF308700FF308800FF3089000313831210
:10002000C1309F000313831600309F000313831217
:100030000313831619309900243098000313831298
:10004000903098001A081A081A08262803138312F9
:1000500000308600A901FE30A200AE210030AA00C7
:10006000A930AB00AC0001303B202918C420A320EC
:100070004520742034288C1E08001A08A400013082
:10008000A9001A081A081A0808002A1C0800A61F46
:100090004C28AC1F5C285E28AC1F4F285A282C081F
:1000A0002602FC3903196E282C082602031C72282C
:1000B000702808003C21080036210800260880131B
:1000C000A1002C0880132102FC3903196E282C088A
:1000D00080132102031C7228702808004D2108009B
:1000E000362108003C2108002A1C0800A71F7B2895
:1000F000AB1F8B288D28AB1F7E2889282B08270251
:10010000FE3903199D282B082702031CA1289F28CC
:100110000800432108004821080027088013A10097
:100120002B0880132102FE3903199D282B08801308
:100130002102031CA1289F28080050210800482103
:1001400008004321080003138312C1309F00FE30D2
:10015000AE211F1500001F19AB281E08A600C930CC
:100160009F00FE30AE211F1500001F19B5281E0884
:10017000A700D1309F00FE30AE211F1500001F19CF
:10018000BF281E08A8000800A901A408A500013086
:100190002506031936210230250603193C210330B8
:1001A0002506031943211E3025060319302104308A
:1001B0002506031948210530250603194D2106306F
:1001C0002506031950211430250603192421153062
:1001D0002506031928211630250603192C21453040
:1001E000250603195621603025060319A2210A307D
:1001F0002506031953216430250603190C216530A7
:100200002506031914216630250603191C216730C1
:1002100025060319102108000130AA00A2210800B8
:100220000030AA00A2210800A2213B20291C152988
:100230002408AC00A2210800A2213B20291C1D2972
:100240002408AB00A221080026089C21A221080056
:1002500027089C21A221080028089C21A22108002F
:1002600026089C2127089C21A2210800BF30860572
:10027000803003108604080003107F30860540306C
:10028000031086040800EF3086052030860408003D
:10029000DF308605103086040800303086050800FF
:1002A000C03086050800003086000800840104087C
:1002B000840A60210038031908009C21572908008E
:1002C0008207533461346C346C3465345434723482
:1002D000613463346B3465347234203431342E34F9
:1002E000303420346234793420344A346134763402
:1002F0006934653472342034413472347234693470
:1003000062346134733420344C34E1347A346134EF
:1003100072346F3420344034323430343034323438
:1003200020344D346F34763469346C3453346F3444
:1003300075346E3464340034000000000C1E9C29B7
:100340009900080045300C1E9C29990008000130D6
:10035000A100A10BA929A20BA82908006430A100C3
:10036000A10BB029A20BAF290800FA30A200AE21E0
:1003700000308600FA30A200AE21FF30860008006F
:02400E00723FFF
:00000001FF
